:020000040000FA
:10000000012885100510051185118316EF30810038
:1000100000308500FF308600831200308B0089019C
:100020000C3084008001840A041F1228041E122848
:10003000831200308B00103091000230900080302D
:100040008F001030940043309300B930920000309C
:100050008E0000308D0092308C002E2811089A00FE
:100060009A0D9A0D9A0D0530A1009A0D0318B92822
:10007000BB28A920A10B3528100899000830A10041
:10008000990D0318BD28BF28A920A10B40280F08EF
:1000900098000830A100980D0318C128C328A92092
:1000A000A10B4B2805150000051114089D009D0D9E
:1000B0009D0D9D0D0530A1009D0D0318C528C72875
:1000C000A920A10B5C2813089C000830A1009C0DFE
:1000D0000318C928CB28A920A10B672812089B0068
:1000E0000830A1009B0D0318CD28CF28A920A10B13
:1000F00072280515000005110E089700970D970D41
:10010000970D0530A100970D0318AD28AF28A92041
:10011000A10B83280D0896000830A100960D031846
:10012000B128B328A920A10B8E280C08950008300F
:10013000A100950D0318B528B728A920A10B99286F
:10014000051500000511000000008515D120640090
:100150002E28051400000510080085148728851036
:100160008728851492288510922885149D2885104B
:100170009D28851439288510392885144428851030
:10018000442885144F2885104F2885146028851031
:10019000602885146B2885106B28851476288510B7
:1001A0007628A00164009F0164009E0164000000A5
:1001B000000000000000061CE4289E0BD7289F0BBF
:1001C000D528A00BD328080085113030A500640085
:1001D000A4016400A3016400A2016400A20BEE2844
:1001E000A30BEC28A40BEA28A50BE82864002E2812
:02400E00F63F7B
:00000001FF
